:100000000C9476070C94BA070C94BA070C94BA07B0
:100010000C94BA070C94BA070C94BA070C94BA075C
:100020000C94BA070C94BA070C9405130C94D713CC
:100030000C94BA070C94BA070C94BA070C94BA073C
:100040000C94BA070C94B12C0C94BA070C94BA0710
:100050000C94BA070C94A9220C94BA070C94BA0712
:100060000C94BA070C94BA070C94BA070C94BA070C
:100070000C94BA070C94BA070C94BA070C94BA07FC
:100080000C94BA070C94BA070C94BA070C94BA07EC
:100090000C94BA070C94BA070C94BA070C94BA07DC
:1000A0000C94BA070C94BA070C94BA07441466145B
:1000B000541566145415AB14CE1454152315361567
:1000C0007D187D18AC18AC18EF182D19461B461B6F
:1000D0004619461B471A471A1A1B461B461B311B5B
:1000E0000147024701470247012102210128022856
:1000F0000001470247014702470120022001280270
:1001000028000147024701470247011F021F01283B
:100110000228000147024701470247011E021E0153
:1001200028022800000001C002C003C004C005C0AE
:10013000018C028C2E004C002900E1003582000069
:100140001E00140004001D0034004D821F001A0020
:1001500015001B00E1042A712000090016000600AA
:1001600050002C7221001300170019004F004A00A4
:1001700022000A00070005000000E20050000254BF
:100180000000007F000001204F00025400000077B3
:100190000000E20023000D000B000E000000E6004E
:1001A00024000F001100100052004B002500180021
:1001B000080036005100287226001C000C00370091
:1001C0002F002B71270033001200387130004E834E
:1001D0002D0031003400E500008200002E004C00AC
:1001E0002900E100358200001E00140004001D00FB
:1001F00034004D821F001A0016001B00E1042A7112
:10020000200008000700060050002C722100150095
:10021000090019004F004A00220017000A000500DB
:100220000000E200500002540000007F00000120A6
:100230004F000254000000770000E20023001C0081
:100240000B0011000000E600240018000D00100053
:1002500052004B0025000C000E00360051002872A1
:10026000260012000F0037002F002B71270013000B
:100270003300387130004E832D0031003400E5002A
:1002800000820000010001000100010001000000E7
:100290003A001E0220022202010001003B001F0260
:1002A00021022302010001003C002F0226022F0040
:1002B000010001003D003002270230000100010072
:1002C0003E0031023500350200000100010001004E
:1002D0000000010000000100010001000000010019
:1002E000000001003F005200510024020000010004
:1002F0004000240021001E000100010041002500F3
:1003000022001F00370001004200260023002000C9
:1003100027000100430025022E0231002E000100BB
:100320004400450001000100010000000000000041
:100330000000000000000000000006200220000075
:100340000000010000000720032000000000010061
:100350000000000004200000000001000000000078
:100360000520000000000100000000000000000067
:10037000000001000000000000000000000001007B
:10038000000000000000000000000100000000006C
:10039000000000000000010000000000000000005C
:1003A000000001000000000000000000000001004B
:1003B000000000000000000000000100000000003C
:1003C000000000000000010000000000000000002C
:1003D000000000000A002530313662003A20002576
:1003E000303258000A722F632030313233343536C0
:1003F0003738394142434445460A000A0025303225
:100400005800626F756E6365213A20006C656674F2
:1004100020736964652061747461636865640A00AF
:100420006C6566742073696465206E6F74207265F4
:1004300073706F6E64696E670A00747279696E67B3
:1004400020746F207265736574206D637032333071
:1004500031380A005B735D004B6579626F617264CD
:100460002073746172742E0A005B575D005B535DEC
:10047000005B525D005B445D005B435D001603451D
:1004800000720067006F0044006F00780020004594
:10049000005A00000016034500720067006F004418
:1004A000006F007800200045005A00000004030996
:1004B0000409028D00050100A0FA090400000103EF
:1004C000010100092111010001223F0007058103FC
:1004D00008000A09040100010301020009211101B9
:1004E0000001224D000705820308000A09040200EA
:1004F0000103000000092111010001223600070557
:10050000830308000A090403000203000000092114
:1005100011010001222000070584032000010705C6
:100520000403200001090404000103000000092164
:100530001101000122390007058503100001120195
:10054000100100000008EDFE071301000102000188
:1005500005010906A101050719E029E71500250194
:100560009508750181020508190129059505750190
:10057000910295017503910105071900297715006E
:100580002501957875018102C00631FF0974A1012A
:100590000975150025FF952075088102097615005B
:1005A00025FF952075089102C005010980A10185EC
:1005B0000216010026B7001A01002AB7007510952F
:1005C000018100C0050C0901A10185031601002667
:1005D0009C021A01002A9C02751095018100C00539
:1005E000010902A1010901A1000509190129051547
:1005F00000250195057501810295017503810105AD
:1006000001093009311581257F9502750881060998
:10061000381581257F950175088106050C0A380279
:100620001581257F950175088106C0C00501090661
:10063000A101050719E029E71500250195087501B5
:1006400081029501750881010508190129059505A3
:10065000750191029501750391010507190029FFA4
:10066000150025FF950675088100C00A0025303267
:100670005820006B6579626F6172645F7265706F9C
:1006800072743A20000A0025303258006B65796296
:100690006F6172645F7365745F6C65643A200064B7
:1006A000656C5F6B65795F6269743A2063616E2780
:1006B000742064656C3A20253032580A0061646405
:1006C0005F6B65795F6269743A2063616E2774209D
:1006D0006164643A20253032580A00646F6E652EDA
:1006E0000A00626F6F676D61676963207363616E93
:1006F0003A202E2E2E2000290A002575002F0025D5
:1007000075005D2800256400200025640020002578
:10071000640020002564007C0025303258006D6F95
:100720007573656B6579205B62746E7C78207920C7
:100730007620685D287265702F61636C293A205BB2
:10074000006D6B5F776865656C5F74696D655F747C
:100750006F5F6D6178203D2025640A006D6B5F77C7
:100760006865656C5F6D61785F7370656564203D79
:100770002025640A006D6B5F74696D655F746F5F3F
:100780006D6178203D2025640A006D6B5F6D617896
:100790005F7370656564203D2025640A006D6B5FA2
:1007A000696E74657276616C203D2025640A006D67
:1007B0006B5F64656C6179203D2025640A006D6B78
:1007C0005F776865656C5F74696D655F746F5F6D99
:1007D0006178203D2025640A006D6B5F7768656550
:1007E0006C5F6D61785F7370656564203D20256482
:1007F0000A006D6B5F74696D655F746F5F6D617822
:10080000203D2025640A006D6B5F6D61785F737019
:10081000656564203D2025640A006D6B5F696E7418
:10082000657276616C203D2025640A006D6B5F6403
:10083000656C6179203D2025640A000A0025750059
:10084000363A20776865656C5F74696D655F746FB3
:100850005F6D61783A20000A00257500353A2077EF
:100860006865656C5F6D61785F73706565643A207B
:10087000000A00257500343A2074696D655F746F55
:100880005F6D61783A20000A00257500333A206DCB
:1008900061785F73706565643A20000A0025750011
:1008A000323A20696E74657276616C286D73293AEC
:1008B00020000A00257500313A2064656C617928B2
:1008C0002A31306D73293A20000A092D2056616CB7
:1008D000756573202D0A004D3E004D25643E2000B5
:1008E0003F007365742064656661756C740A00432B
:1008F0003E200077686572652064656C74613A20FB
:10090000637572736F723D25642C20776865656C22
:100910003D25640A53656520687474703A2F2F650D
:100920006E2E77696B6970656469612E6F72672FCF
:1009300077696B692F4D6F7573655F6B6579730AA6
:10094000000A092D204D6F7573656B6579202D0A9E
:100950004553432F713A09717569740A313A096434
:10096000656C6179282A31306D73290A323A096938
:100970006E74657276616C286D73290A333A096D5D
:1009800061785F73706565640A343A0974696D65EE
:100990005F746F5F6D61780A353A09776865656CD9
:1009A0005F6D61785F73706565640A363A097768D0
:1009B00065656C5F74696D655F746F5F6D61780A02
:1009C0000A703A097072696E742076616C7565738D
:1009D0000A643A097365742064656661756C7473A2
:1009E0000A75703A092B310A646F776E3A092D3116
:1009F0000A706775703A092B31300A7067646F7737
:100A00006E3A092D31300A0A7370656564203D2005
:100A100064656C7461202A206D61785F7370656510
:100A200064202A2028726570656174202F20746903
:100A30006D655F746F5F6D6178290A003F004D3E00
:100A40002000433E20004C25640A000A092D204363
:100A50006F6E736F6C65202D0A4553432F713A09F1
:100A6000717569740A6D3A096D6F7573656B657997
:100A70000A000A092D204D61676963202D0A643A36
:100A80000964656275670A783A096465627567206A
:100A90006D61747269780A6B3A09646562756720E2
:100AA0006B6579626F6172640A6D3A09646562759B
:100AB00067206D6F7573650A763A0976657273699A
:100AC0006F6E0A733A097374617475730A633A0935
:100AD000636F6E736F6C65206D6F64650A302D34C3
:100AE0003A096C61796572302D34284631302D46D3
:100AF00034290A506175733A09626F6F746C6F61C3
:100B00006465720A653A09656570726F6D0A6E3ABE
:100B1000094E4B524F0A7A3A09736C656570204C46
:100B2000454420746573740A000A002575002E6E12
:100B30006B726F3A20000A002575002E7377617082
:100B40005F6261636B736C6173685F6261636B7337
:100B5000706163653A20000A002575002E73776185
:100B6000705F67726176655F6573633A20000A00A3
:100B70002575002E6E6F5F6775693A20000A0025A3
:100B800075002E737761705F72616C745F72677548
:100B9000693A20000A002575002E737761705F6C3A
:100BA000616C745F6C6775693A20000A00257500F6
:100BB0002E636170736C6F636B5F746F5F636F6ED6
:100BC00074726F6C3A20000A002575002E737761ED
:100BD000705F636F6E74726F6C5F636170736C6F64
:100BE000636B3A20000A0025303258006B65796D3E
:100BF00061705F636F6E6669672E7261773A20007D
:100C00000A002575002E6D6F7573653A20000A0085
:100C10002575002E6B6579626F6172643A20000A57
:100C2000002575002E6D61747269783A20000A0003
:100C30002575002E656E61626C653A20000A0025FC
:100C40003032580064656275675F636F6E6669670E
:100C50002E7261773A20000A00257500646566618E
:100C6000756C745F6C617965723A20003F004E4B81
:100C7000524F3A206F66660A004E4B524F3A206F31
:100C80006E0A0074696D65725F636F756E743A20E9
:100C90002530346C580A006B6579626F6172645F4D
:100CA0006E6B726F3A2025580A006B6579626F612E
:100CB00072645F69646C653A2025580A006B657937
:100CC000626F6172645F70726F746F636F6C3A20F1
:100CD00025580A00686F73745F6B6579626F617283
:100CE000645F6C65647328293A2025580A000A0954
:100CF0002D20537461747573202D0A004743433AC5
:100D000020342E392E33204156522D4C4942433A3D
:100D100020312E382E31204156525F415243483AFD
:100D200020617672350A004F5054494F4E533A2095
:100D30004C55464120424F4F544D41474943204D69
:100D40004F5553454B45592045585452414B4559F1
:100D500020434F4E534F4C4520434F4D4D414E4441
:100D6000204E4B524F203531320A004255494C44F7
:100D70003A20333064623330302D646972747920E4
:100D80002830373A35373A3335204A616E203237CA
:100D90002032303136290A005649443A203078460C
:100DA000454544284572676F446F7820455A29208D
:100DB0005049443A20307831333037284572676FD4
:100DC000446F7820455A29205645523A20307830D1
:100DD0003030310A00444553433A20742E6D2E6B57
:100DE0002E206B6579626F617264206669726D771F
:100DF00061726520666F72204572676F646F780A52
:100E0000000A092D2056657273696F6E202D0A0045
:100E10000A6D6F7573653A206F66660A000A6D6F1A
:100E20007573653A206F6E0A000A6B6579626F61AF
:100E300072643A206F66660A000A6B6579626F61B8
:100E400072643A206F6E0A000A6D61747269783AB2
:100E5000206F66660A000A6D61747269783A206FC5
:100E60006E0A000A64656275673A206F6E0A000AAE
:100E700064656275673A206F66660A000A0A626FE7
:100E80006F746C6F616465722E2E2E2000433E20BD
:100E9000006565636F6E6669673A0A00536C656545
:100EA00070204C454420746573740A0000000000F3
:100EB00000000000000000010204060A0F17202CA9
:100EC0003A4A5D71879DB3C7DAE9F5FCFFFCF5E9A5
:100ED000DAC7B39D87715D4A3A2C20170F0A0604C2
:100EE00002010000000000000000000011241FBEED
:100EF000CFEFDAE0DEBFCDBF04B603FE24C08091A1
:100F0000F9019091FA01A091FB01B091FC018730A9
:100F1000904BA740B04BB9F41092F9011092FA012E
:100F20001092FB011092FC0114BE84B7877F84BF2E
:100F300088E10FB6F89480936000109260000FBEB5
:100F4000E0E0FFE3099511E0A0E0B1E0EEEFFCE5A1
:100F500002C005900D92AA33B107D9F711E0AAE3B8
:100F6000B1E001C01D92A93FB107E1F70E943D1019
:100F70000C947D2E0C940000FF93EF93E0913A01C6
:100F8000F0913B01309709F00995EF91FF91089599
:100F9000FC018591803011F0EFDFFBCF0895FF2732
:100FA000E0E230E247FF0CC0419597FF09C0EDE257
:100FB0006095709580959095611D711D811D911DA5
:100FC00027FF02C0219530E350E2AA27660F771F62
:100FD000881F991FAA1FA41710F0A41B63955A9588
:100FE000A9F7AA3008F0A95FA05DAF93F39561154A
:100FF00071058105910541F7ED3211F4EF93F395F9
:10100000F21718F43F93F395FBCF8F91B5DFFA9564
:10101000E1F70895E991F9918591803021F08532C9
:1010200019F0AADFF9CF089520E0E89455915532E0
:10103000C1F3503311F4689455915A3348F4505326
:1010400090F3220F022E220F220F200D250FF4CF36
:101050000EF4219589919991533619F3533729F15B
:10106000533559F1BC0188279927E8945C3621F45F
:101070008991999168945591543639F446EF7EF0F0
:1010800077FF0DC08FEF9FEF0AC055374AE039F068
:10109000583540E121F0523642E009F00895FF93BF
:1010A000EF937DDFEF91FF91B7CFFF93EF93FC01BB
:1010B00081918030B9F360DFFBCFFF93EF9368DF5E
:1010C000F1CFDF93CF93CDB7DEB72596A3DFCF91D6
:1010D000DF910895CF93DF93EC01623039F128F46A
:1010E000662349F0613091F02DC0643029F108F198
:1010F000653029F127C08A81882321F085EE0E947E
:101100001A1720C085EE0E94E2171CC08A8188232E
:1011100051F085EE0E941A1785EE0E94E21783EEC9
:101120000E941A1703C083EE0E94E2178A81882367
:1011300061F08A81882361F08A81882361F08A8145
:10114000882361F080E090E00BC083E191E008C06B
:1011500082E091E005C081EF90E002C080EE90E077
:10116000DF91CF91089580E090E008956091BC01F7
:101170007091BD018091BE019091BF010E94A82194
:1011800056985E9825982D9826982E9827982F98EF
:10119000823019F0833021F00895259A2D9A089510
:1011A000269A2E9A089586EB98E0892B11F00E94DA
:1011B000B60880E090E0089556985E9825982D989E
:1011C00026982E9827982F988FEF90E0909389007B
:1011D0008093880090938B0080938A0090938D0079
:1011E00080938C00259A2D9A2FEF80E792E0215072
:1011F00080409040E1F700C00000269A2E9A2FEF21
:1012000080E792E0215080409040E1F700C000006C
:10121000279A2F9A2FEF80E792E02150804090404C
:10122000E1F700C0000025982D982FEF80E792E0AD
:10123000215080409040E1F700C0000026982E9891
:101240002FEF80E792E0215080409040E1F700C00E
:10125000000027982F9856985E9825982D982698E4
:101260002E9827982F98089589EA8093800089E026
:101270008093810024982C983F988AB18F748AB902
:101280006E98479A8BB1806B8BB9769A0E94DC0876
:1012900083EB98E0892B11F00E94B30880E090E086
:1012A000089580E28093000180913C0181110EC07D
:1012B0000E94A00981E080933C012FEF83ED90E331
:1012C000215080409040E1F700C0000080E40E947F
:1012D000A6098093000181112EC00E94D00980933D
:1012E0000001811128C00E94D00980930001811162
:1012F00022C08FE30E94D0098093000181111BC09E
:101300000E94C80980E40E94A6098093000181110F
:1013100012C08CE00E94D0098093000181110BC0A3
:101320000E94D00980930001811105C08FE30E94C3
:10133000D009809300010E94C8098091000108959E
:101340001092B9008AE08093B800089594EA9093CF
:10135000BC009091BC0097FFFCCF9091B900987FA2
:10136000983021F0903111F081E008958093BB0016
:1013700084E88093BC008091BC0087FFFCCF809103
:10138000B900887F883111F0803471F780E00895CA
:1013900084E98093BC008091BC0084FDFCCF08955B
:1013A0008093BB0084E88093BC008091BC0087FFE1
:1013B000FCCF9091B900987F81E0983209F480E0E9
:1013C000089584E88093BC008091BC0087FFFCCF27
:1013D0008091BB00089580910001811115C080E4C7
:1013E0000E94A6098093000181110CC082E10E9435
:1013F000D00980930001811105C08FEF0E94D009B0
:10140000809300010E94C80984B1807F84B985B1AE
:10141000807F85B98AB1837F8AB98BB1837F8BB98D
:101420003E98469808950E945109809300010E94B9
:10143000EB0980B38C7080BB81B3836F81BBAEE35B
:10144000B1E0ECE4F1E08EE08E0F11921D928E136C
:10145000FCCF84E399E0892B11F00C9434090895B2
:101460009F92AF92BF92CF92DF92EF92FF920F9333
:101470001F93CF93DF93809100018823E1F0809147
:101480003D018F5F80933D01811115C08AE394E097
:101490000E94C8070E94510980930001882329F007
:1014A00080E294E00E94C80706C08CE094E00E94AD
:1014B000C8070E94DC080EE311E0C0E0D0E0BB24C6
:1014C000B39482E0A82ECC24C394D12C2DEFE22E2D
:1014D00023E0F22EC730D10500F580910001811183
:1014E00064C080E40E94A60980930001811112C0AB
:1014F00082E10E94D0098093000181110BC0C601D6
:101500000C2E01C0880F0A94EAF780950E94D0093A
:10151000809300010E94C80948C0CA30A1F028F495
:10152000C83059F0C93061F005C0CC3089F070F096
:10153000CD3089F0209A289810C0219A29980DC0A2
:10154000229A2A980AC0239A2B9807C0529A01C05F
:10155000539A5B9802C03E9A469890EA9A95F1F7A2
:101560009FB1799902C082E001C080E091709B2513
:10157000982B7C9902C084E001C080E0892B7D9982
:1015800002C038E001C030E0832B7E9902C020E128
:1015900001C020E0822B9FB19095991F9927991F38
:1015A0009295990F907E892B10C080910001811136
:1015B00074C080E40E94A60980930001882309F486
:1015C00059C0912C0E94C809892DF8019081981763
:1015D00039F1808380910101882301F18091D70145
:1015E00080FF04C082E094E00E94C8078091D70188
:1015F00080FF0CC0809101011F928F93FF92EF92A8
:101600000E9461080F900F900F900F908091D7016A
:1016100080FF04C08BEF93E00E94C807A0920101F5
:101620000E94EB0921960F5F1F4FCE30D10509F0C4
:1016300051CF809101018823B1F081508093010145
:10164000882339F08FE99FE00197F1F700C000008F
:101650000AC0ACE4B1E0EEE3F1E0CF01825F91912A
:101660009D938E13FCCF83ED98E0892BC1F00E94EF
:10167000D30815C083E10E94D00980930001811135
:10168000A0CF81E40E94A60980930001811199CF27
:101690000E94E109982E909495CF80E096CF81E04A
:1016A000DF91CF911F910F91FF90EF90DF90CF903E
:1016B000BF90AF909F900895E82FF0E0E45BFE4F5D
:1016C00080810895CF92DF92EF92FF920F931F9344
:1016D000CF93DF9384EE93E00E94C8078CE4E82E5A
:1016E00081E0F82EC0E0D0E09FEDC92E93E0D92E26
:1016F00006ED13E0DF93CF93DF92CF920E94610853
:101700008CED93E00E94C807F70181917F0190E082
:101710000E940E229F938F931F930F930E94610844
:1017200084ED93E00E94C80721968DB79EB7089676
:101730000FB6F8949EBF0FBE8DBFCE30D105D1F647
:10174000DF91CF911F910F91FF90EF90DF90CF909D
:1017500008958B3B910578F4883A910540F5853AD8
:101760009105D0F48430910508F0B1C08130910525
:1017700009F4ADC06BC0803E910508F467C0883E97
:10178000910508F4A4C09C01205F31092031310586
:1017900008F05CC090650895853A910509F459C038
:1017A000863A910509F058C082E890E40895883A95
:1017B000910509F454C0893A910509F453C08A3A55
:1017C000910509F452C08B3A910509F451C08C3A45
:1017D000910509F450C08D3A910509F44FC0803B42
:1017E000910509F44EC08E3A910509F44DC08F3A27
:1017F000910509F44CC0813B910509F44BC0823B33
:10180000910509F44AC0833B910509F449C0843B22
:10181000910509F448C0853B910509F447C0863B12
:10182000910509F446C0873B910509F445C0883B02
:10183000910509F444C0893B910509F443C08A3BF2
:10184000910509F442C080E094E4089580E090E0BE
:10185000089581E890E4089583E890E4089582EE85
:1018600094E4089589EE94E408958AEE94E408954A
:1018700085EB94E4089586EB94E4089587EB94E473
:1018800008958CEC94E408958DEC94E4089583E835
:1018900095E408958AE895E4089582E995E4089529
:1018A00084E995E4089581E296E4089583E296E45C
:1018B000089584E296E4089585E296E4089586E228
:1018C00096E4089587E296E408958AE296E40895FE
:1018D000089596E0799FF001112494E5899FE00D29
:1018E000F11D1124E60FF11DEE0FFF1FEC5CFE4F02
:1018F000859194910895880F991FFC01EC55F04053
:10190000859194910895880F991FFC01EC5DFE4F1D
:1019100085919491089526E0729FF001112444E589
:10192000849FE00DF11D1124E60FF11DEE0FFF1F46
:10193000EC5CFE4F859194919C013A9521154FE105
:10194000340708F41AC13F512115304120F49F702B
:101950000E94830C08959C0130532115304118F4E6
:101960009927906C0895811520E5920769F40E94EB
:10197000681B4FEF84E39CE0415080409040E1F7CA
:1019800000C000000C94CE22813020E5920731F493
:101990008091D70181608093D70108959C013055D3
:1019A0002115304108F051C0292F33272F703327DC
:1019B00021303105D9F4AC014370552702C0220F04
:1019C000331F4A95E2F73C68AC0164E0440F551FB1
:1019D0006A95E1F744275370242B352B73E0880F69
:1019E000991F7A95E1F7807699271DC0223031053D
:1019F00029F4982F8827816F906A08952330310544
:101A0000A9F4AC014370552721E030E002C0220F59
:101A1000331F4A95E2F73C6843E0880F991F4A95C7
:101A2000E1F7807E9770822B932B08952430310547
:101A3000E1F4AC014370552721E030E002C0220FF1
:101A4000331F4A95E2F73A68E7CF9C0130572115DA
:101A5000304118F49F70906208959C013058211510
:101A6000304118F49F70906A0895803E9105E0F42B
:101A7000803C910558F58133910509F46FC048F415
:101A80008932910509F463C08A32910509F46DC069
:101A900072C089339105E9F082389105D1F0853320
:101AA000910509F44DC067C0833E910581F138F47A
:101AB000803E9105B9F0823E9105D9F05CC0863E2A
:101AC000910561F1873E9105A1F155C00E947B0C03
:101AD00008952091EA0120FD02C021FF4CC080EE54
:101AE00090E049C08091EA0180FFF9CF89E390E05E
:101AF00042C08091EA0182FF0EC08091EA0184FF1A
:101B000003C080E090E037C083EE90E034C0809165
:101B1000EA0182FFF2CF82EE90E02DC08091EA01CF
:101B200083FF0BC08091EA0184FDEBCF87EE90E04C
:101B300022C08091EA0183FFF5CF86EE90E01BC0C2
:101B40008091EA0185FF07C089E290E014C080918E
:101B5000EA0185FFF9CF85E390E00DC08091EA01AD
:101B600086FF07C08AE290E006C08091EA0186FF06
:101B7000F9CF81E390E00E94A90B08950895809128
:101B80006D0108959FB7F89410925C019FBF9091EA
:101B9000F001943009F057C09091E9009F703091A6
:101BA000EC00232F217030FD20E8922B24E02093BD
:101BB000E9002091EB0020FF43C02091EE0027FFB9
:101BC0003FC020915A01222321F02091E80025FFF7
:101BD00037C010925A0126E03091E80035FD15C05B
:101BE0003091F001343061F53091EB0035FD28C0C3
:101BF000215021F481E080935A0122C0EFE9FFE0F7
:101C00003197F1F700C00000E7CF8093F100809199
:101C1000E80085FD0AC08091E80080FFFCCF80913C
:101C2000E8008E778093E80006C08FB7F89421E033
:101C300020935C018FBF9F709093E90080E008952E
:101C40009F709093E9008FEF0895CF93DF9300D0BA
:101C50001F92CDB7DEB79C018091F001843019F559
:101C600093E099833B832A839093E9008FEF9091CF
:101C7000E800815095FD06C095ED9A95F1F70000BA
:101C80008111F5CF8091E80085FF0DC040E050E064
:101C900063E070E0CE0101960E94F5108091E800AB
:101CA0008E778093E8000F900F900F90DF91CF9187
:101CB0000895CF93DF9300D01F92CDB7DEB7209168
:101CC000F001243021F522E029839B838A8383E07D
:101CD0008093E9008FEF9091E800815095FD06C058
:101CE00095ED9A95F1F700008111F5CF8091E8000C
:101CF00085FF0DC040E050E063E070E0CE0101964A
:101D00000E94F5108091E8008E778093E8000F9094
:101D10000F900F90DF91CF9108952091F001243022
:101D2000F1F422E02093E9002FEF3091E8002150F8
:101D300035FD06C035ED3A95F1F700002111F5CFDC
:101D40002091E80025FF0BC040E050E065E070E026
:101D50000E94F5108091E8008E778093E800089546
:101D6000CF93DF932091F001243009F048C0EC01BB
:101D700080910C018823E1F080910D018823C1F04E
:101D800085E08093E9008FEF9091E800815095FD08
:101D900006C095E19A95F1F700008111F5CF809189
:101DA000E80085FF2CC040E050E060E170E017C023
:101DB00081E08093E9008FEF9091E800815095FDDC
:101DC00006C095ED9A95F1F700008111F5CF80914D
:101DD000E80085FF14C040E050E068E070E0CE010C
:101DE0000E94F5108091E8008E778093E80080E1F2
:101DF000FE01ADE5B1E001900D928A95E1F7DF912A
:101E0000CF91089589E794E00E94C8078091EF017F
:101E1000811109C00E948A120E94E7128091E2009B
:101E200084608093E200089585E794E00E94C807EB
:101E30001092EF01089581E794E00C94C8078DE6B5
:101E400094E00E94C8070C949E2C89E694E00E94BE
:101E5000C8070E9464220E94A42C0E948C150C9436
:101E6000BE0D20915B012F5F822F62E30E94122E34
:101E7000992319F020935B01089510925B018091E2
:101E80005C01882371F18091F001843041F58091EB
:101E9000E9008F702091EC00922F917020FD90E866
:101EA000892B94E09093E9009091EB0090FF14C08F
:101EB0009091EE0097FF10C09091E80095FF03C04D
:101EC0001092F100F9CF9091E80090FF05C0909139
:101ED000E8009E779093E8008F708093E90010925D
:101EE0005C01089542E061EC81E00E94041242E04E
:101EF00061EC82E00E94041242E061EC83E00E9407
:101F0000041242E261EC84E00E94041242E161ECBE
:101F100085E00C9404128091F201833009F455C0DD
:101F200030F4813071F0823009F48EC008958A3027
:101F300009F47AC08B3009F460C0893009F09CC084
:101F400020C08091F101813A09F096C08091E800AB
:101F5000877F8093E8008091F5019091F601892BAD
:101F600021F460E18DE591E003C060E080E090E065
:101F700070E00E9440118091E8008B778093E80028
:101F800008958091F101813209F076C08091F501C8
:101F90009091F601009719F0049709F06DC08091B7
:101FA000E800877F8093E8008091E80082FD05C00B
:101FB0008091F0018111F8CF5FC08091F100809392
:101FC0006D018091E8008B7753C08091F101813AD7
:101FD00009F052C08091F5019091F601892B09F02A
:101FE0004BC08091E800877F8093E8008091E800F3
:101FF00080FFFCCF80910C0136C08091F1018132CD
:10200000D9F58091F5019091F601892BA9F5809180
:10201000E800877F8093E8000E9439128091F301E5
:1020200080930C010C94681B8091F101813221F5A1
:102030008091E800877F8093E8000E9439128091A8
:10204000F40180936E0108958091F101813AA1F429
:102050008091E800877F8093E8008091E80080FF0E
:10206000FCCF80916E018093F1008091E8008E7723
:102070008093E8000C943912089584B7877F84BF59
:1020800088E10FB6F89480936000109260000FBE54
:1020900090E080E80FB6F89480936100909361001F
:1020A0000FBE0E9419160E948A120E94E7128091A8
:1020B000E20084608093E20082EC9DE00E94A32114
:1020C00078940E946C150E941B1682E091E00E9499
:1020D00087150E948C2C88E594E00E94C8078091A7
:1020E000F001853089F484E594E00E94C8070E94DD
:1020F00028228091EE01882391F30E9450228823A8
:1021000071F30E94DF10EBCF0E944916E8CF292F10
:10211000332723303105C9F064F42130310581F0D3
:102120002230310509F043C08DE890E021EB34E026
:1021300042C021323105F1F02232310541F137C080
:1021400082E190E02EE335E036C099278130910599
:1021500041F08230910541F0892B49F5EDEAF4E038
:1021600005C0E5E9F4E002C0EDE7F4E0849190E019
:102170009F0121C06530D8F4E62FF0E0EE0FFF1F7D
:10218000EB5DFE4F2081318189E090E014C0653025
:1021900070F470E0FB01EE0FFF1FE55EFE4F208143
:1021A0003181FB01EA5EFE4F808190E004C080E057
:1021B00090E020E030E0FA0131832083089580E14F
:1021C00089BD82E189BD09B400FEFDCF8091D800B0
:1021D0008F7D8093D8008091E00082608093E00042
:1021E0008091E00081FDFCCF0895CF92DF92EF92C5
:1021F000FF920F931F93CF93DF93EC018B016A0142
:102200000E945812811133C0C114D10439F0F60173
:1022100080819181081B190BC80FD91FE12CF12C6B
:102220000115110519F18091E80085FD16C0809116
:10223000E8008E778093E800C114D10449F0F601DC
:1022400080819181E80EF91EF182E08285E00FC065
:102250000E945812882321F30AC089918093F100CB
:1022600001501109FFEFEF1AFF0ADACF80E0DF918A
:10227000CF911F910F91FF90EF90DF90CF90089535
:102280002091F7013091F8012617370748F06115C2
:10229000710539F42091E8002E772093E80001C001
:1022A000B90140E061157105A9F12091F0012223E7
:1022B00009F443C0253009F442C02091E80023FD11
:1022C00040C02091E80022FD32C02091E80020FFAC
:1022D000E9CF4091F3002091F20030E0342BFC0173
:1022E000CF016115710559F02830310540F4819115
:1022F0008093F100615071092F5F3F4FF1CF41E0B2
:102300002830310509F040E02091E8002E77209335
:10231000E800C8CF4111C9CF0AC08091F0018823DD
:1023200061F0853061F08091E80083FD0AC0809102
:10233000E80082FFF2CF80E0089582E0089583E014
:10234000089581E008952091F7013091F801261752
:10235000370748F06115710539F42091E8002E77B0
:102360002093E80001C0B901FC0120E0611571056E
:1023700091F18091F001882309F440C0853009F47F
:102380003FC08091E80083FD3DC08091E80082FD60
:102390002FC08091E80080FFE9CF2091F300809169
:1023A000F20090E0922B6115710559F0883091058B
:1023B00040F424912093F100319661507109019607
:1023C000F2CF21E0089709F020E08091E8008E77B5
:1023D0008093E800CBCF2111CCCF0AC08091F001CF
:1023E000882361F0853061F08091E80083FD0AC0A8
:1023F0008091E80082FFF2CF80E0089582E00895A6
:1024000083E0089581E00895982F973058F59093D0
:10241000E900981739F07091EC002091ED0050918F
:10242000F00003C0242F762F50E021FF19C0309117
:10243000EB003E7F3093EB003091ED003D7F309319
:10244000ED003091EB0031603093EB007093EC00C5
:102450002093ED005093F0002091EE0027FF07C07D
:102460009F5FD3CF8F708093E90081E0089580E073
:1024700008958091F10187FF11C08091E80082FDED
:1024800005C08091F0018111F8CF11C08091E80062
:102490008B770BC08091F001882349F08091E80090
:1024A00080FFF8CF8091E8008E778093E800089550
:1024B0002091E4003091E50095E64091EC00842FF6
:1024C000817040FF22C08091E80080FD1CC0809197
:1024D000F001882391F0853091F08091EB0085FD2B
:1024E00010C04091E4005091E5004217530729F3D2
:1024F0009A01915011F784E0089582E0089583E0F5
:10250000089581E0089580E008954091E80042FF39
:10251000DECF08950E94F8120E940013E0EEF0E072
:10252000808181608083E8EDF0E080818F77808317
:1025300019BCA7EDB0E08C918E7F8C9380818F7E4B
:1025400080831092EF0108950F931F93CF93DF9331
:102550000E94F8120E940013C8EDD0E088818F77A6
:10256000888388818068888388818F7D888319BC6F
:102570001092F0011092EC011092EE011092ED0118
:1025800000EE10E0F80180818B7F8083888181607C
:10259000888342E060E080E00E940412E1EEF0E017
:1025A00080818E7F8083E2EEF0E080818160808395
:1025B000808188608083F80180818E7F808388811C
:1025C00080618883DF91CF911F910F910895E8ED8D
:1025D000F0E080818F7E8083E7EDF0E08081816094
:1025E000808384E082BF81E08093EF010C94A41289
:1025F000E8EDF0E080818E7F80831092E200089504
:102600001092DA001092E10008951F920F920FB617
:102610000F9211242F933F934F935F936F937F9368
:102620008F939F93AF93BF93EF93FF938091E100BC
:1026300082FF0BC08091E20082FF07C08091E10021
:102640008B7F8093E1000E94310F8091DA0080FF40
:102650001FC08091D80080FF1BC08091DA008E7F60
:102660008093DA008091D90080FF0DC080E189BDA0
:1026700082E189BD09B400FEFDCF81E08093F001C5
:102680000E94020F05C019BC1092F0010E94140FA5
:102690008091E10080FF19C08091E20080FF15C0A9
:1026A0008091E2008E7F8093E2008091E200806161
:1026B0008093E2008091D80080628093D80019BC9A
:1026C00085E08093F0010E941F0F8091E10084FF5C
:1026D00030C08091E20084FF2CC080E189BD82E19E
:1026E00089BD09B400FEFDCF8091D8008F7D809315
:1026F000D8008091E1008F7E8093E1008091E2001C
:102700008F7E8093E2008091E20081608093E200FE
:102710008091EC01882311F084E007C08091E300F0
:1027200087FD02C081E001C083E08093F0010E9438
:10273000250F8091E10083FF29C08091E20083FF93
:1027400025C08091E100877F8093E10082E0809343
:10275000F0011092EC018091E1008E7F8093E10006
:102760008091E2008E7F8093E2008091E2008061A0
:102770008093E20042E060E080E00E9404128091D9
:10278000F00088608093F0000E941B0FFF91EF9192
:10279000BF91AF919F918F917F916F915F914F9179
:1027A0003F912F910F900FBE0F901F9018951F9281
:1027B0000F920FB60F9211242F933F934F935F9375
:1027C0006F937F938F939F93AF93BF93CF93DF9339
:1027D000EF93FF93C091E900CF708091EC00D82F68
:1027E000D17080FDD0E81092E9008091F000877FE1
:1027F0008093F00078940E941B141092E90080915D
:10280000F00088608093F000CD2BCF70C093E9007A
:10281000FF91EF91DF91CF91BF91AF919F918F91F8
:102820007F916F915F914F913F912F910F900FBECC
:102830000F901F9018951F93CF93DF93CDB7DEB7FE
:10284000AA970FB6F894DEBF0FBECDBFE1EFF1E05F
:1028500088E08E0F9091F10091938E13FBCF0E9430
:102860008B0F8091E80083FF1FC18091F10190914F
:10287000F201492F50E04A30510508F015C1FA0124
:10288000EA5AFF4F0C94322E803881F0823809F0DA
:102890000BC18091F5018F708093E9008091EB006E
:1028A00085FB882780F91092E90006C08091ED0130
:1028B0009091EE01911182609091E800977F909342
:1028C000E8008093F1001092F100C8C0282F2D7FFE
:1028D00009F0EAC0882319F0823061F0E5C08091E8
:1028E000F301813009F0E0C0933009F080E080937B
:1028F000EE012BC08091F301811127C08091F50179
:102900008F7009F4D1C08093E9002091EB0020FF83
:102910001CC0933021F48091EB00806214C0909130
:10292000EB0090619093EB0021E030E0A90102C040
:10293000440F551F8A95E2F74093EA001092EA008F
:102940008091EB0088608093EB001092E900809109
:10295000E800877F86C08111A7C01091F3011F771F
:102960008091E3008078812B8093E3008091E800E0
:10297000877F8093E8000E9439128091E80080FFF1
:10298000FCCF8091E30080688093E300111102C0C6
:1029900082E001C083E08093F00186C080588230DD
:1029A00008F082C08091F3019091F4018C3D53E0D6
:1029B000950779F583E08A838AE289834FB7F89493
:1029C000DE01139620E03EE051E2E32FF0E0509369
:1029D0005700E49120FF03C0E295EF703F5FEF7076
:1029E0008E2F90E0EA3010F0C79601C0C0968D930C
:1029F0009D932F5F243149F74FBF8091E800877F77
:102A00008093E8006AE270E0CE0101960E944011D6
:102A100014C0AE014F5F5F4F6091F5010E948710B7
:102A2000BC01892B09F440C09091E800977F9093F6
:102A3000E80089819A810E94A3118091E8008B7738
:102A40008093E80031C0803879F58091E800877F75
:102A50008093E8008091EC018093F1008091E80080
:102A60008E778093E8000E9439121EC081111CC02D
:102A70009091F3019230C0F48091E800877F8093B9
:102A8000E8009093EC010E9439128091EC018111D1
:102A900006C08091E30087FD02C081E001C084E0B0
:102AA0008093F0010E94720F8091E80083FF0AC0BA
:102AB0008091E800877F8093E8008091EB0080623E
:102AC0008093EB00AA960FB6F894DEBF0FBECDBF81
:102AD000DF91CF911F910895CF938091F0018823CA
:102AE000A1F0C091E900CF709091EC00892F817026
:102AF00090FD80E8C82B1092E9008091E80083FDEA
:102B00000E941B14CF70C093E900CF910895909359
:102B10007401809373010895E0917301F091740141
:102B2000309721F00190F081E02D099480E0089524
:102B3000EF92FF920F931F93CF93DF93E091730176
:102B4000F09174013097B1F18C010280F381E02D96
:102B500009958091D70182FF2DC080FF04C083E7D3
:102B600096E00E94C807E80110E18DE6E82E86E0B5
:102B7000F82E8091D70180FF0BC088811F928F9320
:102B8000FF92EF920E9461080F900F900F900F90AC
:102B9000115021961111EDCF8091D70180FF0AC00D
:102BA0008BE696E0DF91CF911F910F91FF90EF9010
:102BB0000C94C807DF91CF911F910F91FF90EF9078
:102BC0000895E0917301F0917401309721F0048031
:102BD000F581E02D099408952091710130917201E1
:102BE0008217930771F09093720180937101E091C5
:102BF0007301F0917401309721F00680F781E02D88
:102C00000994089520916F01309170018217930704
:102C100071F09093700180936F01E0917301F091D6
:102C20007401309721F00084F185E02D0994089516
:102C300008950C9418160E946A220E94130A0C949C
:102C40003023CF93C82F8091D70182FF1EC080FF11
:102C500004C08CE896E00E94C8078091D70180FFED
:102C60000CC01F92CF9387E896E09F938F930E94AA
:102C700061080F900F900F900F908091D70180FF07
:102C800004C085E896E00E94C8078C2FCF910C9471
:102C9000BE0DCF92DF92EF92FF920F931F93CF93CF
:102CA000DF93CDB7DEB72B970FB6F894DEBF0FBE1C
:102CB000CDBF0E94300A86E7C82E81E0D82E00E002
:102CC00010E0E02E802F0E945C0BF60141916F0115
:102CD000F42EF826B1F40F5F1F4F0E30110589F75F
:102CE0008FEF89838A831B820E9473228160782FF1
:102CF0009D838C8349815A816B818D810E94EC1662
:102D000040C09091D70191FF04C08B870E94620B55
:102D10008B8520E030E04F2D50E0922FBA01022E3B
:102D200002C0759567950A94E2F760FF24C02E8370
:102D3000EF8221E030E0690102C0CC0CDD1C9A95E5
:102D4000E2F790E08C219D21892B09F420E028876F
:102D50000E9473228160782F9A8789874E815F81D4
:102D600068858A850E94EC16F801EA58FE4F80813A
:102D7000C826C08206C02F5F3F4F2630310569F656
:102D8000AACF0E94A126109175010E948C151817D8
:102D9000A1F00E948C15809375012B960FB6F894C4
:102DA000DEBF0FBECDBFDF91CF911F910F91FF907E
:102DB000EF90DF90CF900C9421162B960FB6F894DD
:102DC000DEBF0FBECDBFDF91CF911F910F91FF905E
:102DD000EF90DF90CF900895CF93DF93CDB7DEB71C
:102DE0002B970FB6F894DEBF0FBECDBF4F83588729
:102DF00069877A878B87DE01119686E0FD01119243
:102E00008A95E9F785E0FE01379601900D928A9543
:102E1000E1F749815A816B817C818D819E810E947D
:102E2000021E2B960FB6F894DEBF0FBECDBFDF910A
:102E3000CF910895CF93882309F4C2C0C82F823858
:102E400059F40E948C1581FDBBC089E30E949E202D
:102E50000E947D2189E30CC0833879F40E948C158F
:102E600080FDAEC083E50E949E200E947D2183E507
:102E70000E94F120CF910C947D21843859F40E9456
:102E80008C1582FD9DC087E40E949E200E947D21BA
:102E900087E4EECF8CEF8C0F813A48F48C2F0E94A0
:102EA000342B81118DC08C2F0E949E20E3CF80E2B5
:102EB0008C0F883048F4C77081E001C0880FCA9534
:102EC000EAF70E944621D6CF8BE58C0F833078F449
:102ED000C53A29F0C63A31F083E890E005C081E8B0
:102EE00090E002C082E890E0CF910C94EC1588E568
:102EF0008C0F833108F064C0C83A39F1C93A41F106
:102F0000CA3A49F1CB3A51F1CC3A59F1CD3A61F193
:102F1000C03B69F1CE3A71F1CF3A79F1C13B81F111
:102F2000C23B89F1C33B91F1C43B99F1C53BA1F18F
:102F3000C63BA9F1C73BB1F1C83BB9F1C93BC1F1EF
:102F4000CA3BC9F180E090E038C082EE90E035C025
:102F500089EE90E032C08AEE90E02FC085EB90E0E1
:102F60002CC086EB90E029C087EB90E026C08CEC6B
:102F700090E023C08DEC90E020C083E891E01DC07C
:102F80008AE891E01AC082E991E017C084E991E0F3
:102F900014C081E292E011C083E292E00EC084E2AC
:102FA00092E00BC085E292E008C086E292E005C0A4
:102FB00087E292E002C08AE292E0CF910C9402167E
:102FC000CF910895882309F44BC0823859F40E94A8
:102FD0008C1581FF45C089E30E949E200E947D21BF
:102FE00089E30CC0833871F40E948C1580FF38C0CF
:102FF00083E50E949E200E947D2183E50E94F120AE
:103000000C947D21843859F40E948C1582FF28C0CD
:1030100087E40E949E200E947D2187E4EFCF9CEFF1
:10302000980F913A58F390E2980F983050F48770C7
:1030300091E001C0990F8A95EAF7892F0E944C21EF
:10304000DFCF9BE5980F933020F480E090E00C9464
:10305000EC15885A833120F480E090E00C9402163D
:103060000895882321F00E9446210C947D21089523
:10307000882321F00E944C210C947D210895BF9259
:10308000CF92DF92EF92FF920F931F93CF93DF9334
:1030900000D000D000D0CDB7DEB725E0FC01DE01C6
:1030A000119601900D922A95E1F7FC014081318142
:1030B0000281258122952F7063817481672B09F429
:1030C000E5C23F3F19F44F3F09F4E0C27C01498358
:1030D0003A8389819A812E830E945D20182FB92E10
:1030E0000E945C200E94231FEB2DE295EF70F0E020
:1030F000E05AFF4F2E810C94322E8B2D807F9B2D1A
:103100009F70F92E882319F0F29480EFF8220023A3
:1031100049F0FF2009F467C28F2D0E9456210E94BA
:103120007D2161C2812F0E94E217FF2009F4AEC207
:103130008F2D0E945C2126960FB6F894DEBF0FBE3D
:10314000CDBFDF91CF911F910F91FF90EF90DF9056
:10315000CF90BF900C947D213B2D307F8B2D8F70B5
:10316000303211F08295807F112319F0113021F156
:103170002CC00023B9F0222309F4A0C1213009F0AA
:103180009DC126960FB6F894DEBF0FBECDBFDF916E
:10319000CF911F910F91FF90EF90DF90CF90BF9054
:1031A0000C946621222319F0213009F46FC28E831A
:1031B0000E9469218E8196C1002321F0223008F0FF
:1031C00065C27CC1211162C28DC1002321F022237E
:1031D00009F474C108C2222309F484C119C22B2D39
:1031E00026952695237030E02115310521F02130F8
:1031F0003105D1F04BC2002321F0812F9B2D93701C
:1032000002C080E090E026960FB6F894DEBF0FBEB5
:10321000CDBFDF91CF911F910F91FF90EF90DF9085
:10322000CF90BF900C94EC15002321F0812F9B2DA3
:10323000937002C080E090E026960FB6F894DEBF4F
:103240000FBECDBFDF91CF911F910F91FF90EF90F7
:10325000DF90CF90BF900C940216812F002319F0BD
:103260000E94272502C00E948F2526960FB6F8944B
:10327000DEBF0FBECDBFDF91CF911F910F91FF90A9
:10328000EF90DF90CF90BF900C9414268B2D83701D
:1032900009F07BC00111FAC1812F82958695877054
:1032A000880F880F912F9F70C92ED12CE12CF12C03
:1032B000082E04C0CC0CDD1CEE1CFF1C0A94D2F7B7
:1032C00014FF12C04FE050E060E070E004C0440F13
:1032D000551F661F771F8A95D2F7CB01BA016095FB
:1032E00070958095909503C060E070E0CB012B2D28
:1032F000269526952370422F50E042305105D9F093
:103300004330510569F16C297D298E299F2941306F
:10331000510551F126960FB6F894DEBF0FBECDBF12
:10332000DF91CF911F910F91FF90EF90DF90CF90A1
:10333000BF900C944A1F6C297D298E299F292696BF
:103340000FB6F894DEBF0FBECDBFDF91CF911F91B6
:103350000F91FF90EF90DF90CF90BF900C94661F7D
:103360000E944A1FC701B60126960FB6F894DEBF29
:103370000FBECDBFDF91CF911F910F91FF90EF90C6
:10338000DF90CF90BF900C942E1F002319F08B2D4F
:10339000817001C08695882309F478C1812F8295B8
:1033A00086958770880F880F912F9F70C92ED12C1A
:1033B000E12CF12C082E04C0CC0CDD1CEE1CFF1CF3
:1033C0000A94D2F714FF12C04FE050E060E070E0C2
:1033D00004C0440F551F661F771F8A95D2F7CB0193
:1033E000BA01609570958095909503C060E070E09B
:1033F000CB012B2D269526952370422F50E042308D
:103400005105D9F04330510569F16C297D298E2988
:103410009F294130510551F126960FB6F894DEBF31
:103420000FBECDBFDF91CF911F910F91FF90EF9015
:10343000DF90CF90BF900C9424206C297D298E2999
:103440009F2926960FB6F894DEBF0FBECDBFDF9141
:10345000CF911F910F91FF90EF90DF90CF90BF9091
:103460000C9440200E942420C701B60126960FB676
:10347000F894DEBF0FBECDBFDF91CF911F910F91AA
:10348000FF90EF90DF90CF90BF900C940820103FFA
:10349000D1F118F4103E50F4A1C0123F09F463C0FA
:1034A00008F44CC0133F09F473C098C01F708B2DF3
:1034B0008F710023A1F00E94A11F812F26960FB6C5
:1034C000F894DEBF0FBECDBFDF91CF911F910F915A
:1034D000FF90EF90DF90CF90BF900C9431180E9436
:1034E000C21F812F26960FB6F894DEBF0FBECDBF48
:1034F000DF91CF911F910F91FF90EF90DF90CF90D0
:10350000BF900C9438180023A9F02111BFC08B2D57
:103510008F7126960FB6F894DEBF0FBECDBFDF9138
:10352000CF911F910F91FF90EF90DF90CF90BF90C0
:103530000C94E71F223008F0A9C0E9CF0023A9F0BE
:103540008B2D8F7126960FB6F894DEBF0FBECDBFC0
:10355000DF91CF911F910F91FF90EF90DF90CF906F
:10356000BF900C94A11F002359F38B2D8F712696C9
:103570000FB6F894DEBF0FBECDBFDF91CF911F9184
:103580000F91FF90EF90DF90CF90BF900C94C21FEF
:10359000002399F08B2D8F7126960FB6F894DEBF1D
:1035A0000FBECDBFDF91CF911F910F91FF90EF9094
:1035B000DF90CF90BF900C948C1F26960FB6F89496
:1035C000DEBF0FBECDBFDF91CF911F910F91FF9056
:1035D000EF90DF90CF90BF900C94821F0023A9F052
:1035E000222309F4ADCF812F26960FB6F894DEBFC3
:1035F0000FBECDBFDF91CF911F910F91FF90EF9044
:10360000DF90CF90BF900C941A17222309F4ADCF0E
:10361000812F26960FB6F894DEBF0FBECDBFDF9187
:10362000CF911F910F91FF90EF90DF90CF90BF90BF
:103630000C94E2174B2D4F70612FC7010E946A084E
:1036400026960FB6F894DEBF0FBECDBFDF91CF91A7
:103650001F910F91FF90EF90DF90CF90BF900C944F
:10366000A61E4B2D4F70612FC70126960FB6F894FA
:10367000DEBF0FBECDBFDF91CF911F910F91FF90A5
:10368000EF90DF90CF90BF900C94680C26960FB609
:10369000F894DEBF0FBECDBFDF91CF911F910F9188
:1036A000FF90EF90DF90CF90BF9008950E9463212C
:1036B0000E9438210E947D210E9447270E941426E3
:1036C00080E090E00E94EC1580E090E00C940216FF
:1036D0000E9453210C94561B0E945D20292F229595
:1036E0002F7030E02C3031054CF42A3031056CF469
:1036F000225031092230310588F407C02C303105C1
:1037000049F02F30310531F009C0803E48F0803F4C
:1037100029F406C093FB882780F9089580E0089576
:1037200081E00895CF93DF9300D000D01F92CDB7F2
:10373000DEB70F900F900F900F900F90DF91CF9109
:103740000895CF93DF9300D000D000D0CDB7DEB77F
:1037500026960FB6F894DEBF0FBECDBFDF91CF9196
:1037600008951F93CF93DF93C091840116E0809159
:103770008501C81799F0D0E01C9FF0011D9FF00D46
:103780001124EA57FE4F4081518162817381848107
:1037900095810E94A11B2196C770E9CFDF91CF913F
:1037A0001F9108954091B6015091B7016091B80101
:1037B0007091B9018091BA019091BB010C94A11B49
:1037C0008091BB0182958F7009F054C08091B8013F
:1037D000882309F44FC080918401A09185016091F4
:1037E000B6017091B7014091B9015091BA01B6E0AC
:1037F0008A1709F43FC090E041155105C1F17F3FA0
:1038000011F46F3FA1F1B89FF001B99FF00D1124A1
:10381000EA57FE4F218172132AC02081621327C00C
:103820002281211124C0238134812417350710F40B
:1038300021503109241B350B283C3105C0F420915F
:10384000BB012F7020612093BB0126E0289FF0016F
:10385000299FF00D1124E557FE4F80818F70806104
:10386000808386EB91E00E943F180C94B11B019677
:103870008770BECF0895CF92DF92EF92FF920F93A1
:103880001F93CF93DF93CDB7DEB762970FB6F8944F
:10389000DEBF0FBECDBF8C0185E0F801DE011D96B5
:1038A00001900D928A95E1F7D8014C9111965C91A7
:1038B000119712966C9112971396CD90DC901497F5
:1038C0003091B6017091B7018091B9019091BA0120
:1038D000009709F46BC17F3F19F43F3F09F466C1BB
:1038E000E090B801EE2009F4C0C02091BB01C816D9
:1038F000D90628F0F601E81BF90BCF0104C080952A
:1039000090958C0D9D1DFF24F394883C910578F0D3
:10391000F12C207F09F0C6C07C2DD98AC88A8989FC
:103920000E94921B86EB91E00E943F18B1C0822F4B
:10393000807F09F046C0751314C0341312C06111A2
:1039400010C02F7020612093BB010E94D21B86EB18
:1039500091E00E943F188091BB01D80115968C938D
:103960002EC0CD2819F15F3F11F44F3FF9F0F62E2C
:1039700061111CC0809184012091850136E082177D
:1039800009F45AC090E0389FF001399FF00D1124DE
:10399000EA57FE4F7181571306C07081471303C069
:1039A0007281711103C001968770E9CFF62E6623EC
:1039B00009F418C18091BB0181608093BB01F12C97
:1039C00011C1751308C0341306C0611104C0809181
:1039D000BB01D801C3C04D875E878D859E856A8BEC
:1039E0000E946C1B6A898823E1F16623D1F1209142
:1039F000BB01822F82958F7090E0029774F08091C6
:103A0000B6019091B70198878F831986DB86CA86A5
:103A10002C87CE0107960E943F1886E0F801A6EB9E
:103A2000B1E001900D928A95E1F70E94E01B0E949F
:103A3000D21BFF24F394D6C04D875E878D859E856B
:103A40000E945D20292F22952F7030E02230310511
:103A50000CF0BCC09F7009F0B6C0805E883008F4DE
:103A6000C1C0C8010E943F18E4CFC816D90608F4A7
:103A700053C0F601E81BF90BCF01883C910508F40F
:103A800050C0F12C7C2DD98AC88A89890E94921B4A
:103A9000E6EBF1E086E0DF011D928A95E9F70E94EE
:103AA000D21BA0C0751314C0341312C0611110C012
:103AB0008091BB01F8018583C8010E943F1886E010
:103AC000E6EBF1E0DF011D928A95E9F7FE2C8AC052
:103AD0004D875E878D859E856A8B0E946C1B6A89E7
:103AE000882309F4BECF662309F4BBCF2091BB0124
:103AF000822F82958F7090E002970CF48ECF809188
:103B0000B6019091B7019A8389831B82DD82CC82B2
:103B10002E83CE0101967FCF809590958C0D9D1DB3
:103B2000ACCFF62E662309F49CCF75132EC0341348
:103B30002CC02091BB0120FD1FC0822F82958F7069
:103B4000D9F0D80115962C9315978F3049F08F5FD7
:103B5000982F9295907F822F8F70892B15968C933A
:103B6000C8010E943F1886E0F801A6EBB1E0019081
:103B70000D928A95E1F793CF86E0F801A6EBB1E0CC
:103B800001900D928A95E1F72DC04D875E878D8556
:103B90009E850E946C1B811140CF8091BB0181608A
:103BA0008093BB01C8010E943F181CC0662309F422
:103BB00058CF4D875E878D859E850E946C1B88231C
:103BC00009F44FCF2ACF811148CF0CC024303105E2
:103BD0000CF047CF9F7009F440CFF8019581907F9A
:103BE00009F03BCF8F2D62960FB6F894DEBF0FBE63
:103BF000CDBFDF91CF911F910F91FF90EF90DF909C
:103C0000CF9008951F93CF93DF93CDB7DEB72C9756
:103C10000FB6F894DEBF0FBECDBF4F8358876987BC
:103C20007A878B879C87CE0107960E943B1C88234E
:103C300069F08F8198852A853B85232BF1F19F3F81
:103C400009F063C08F3F09F060C037C086E0FE0115
:103C50003796DE01119601900D928A95E1F76F81FA
:103C60007885EA85FB85309741F17F3F11F46F3FFE
:103C700021F12091850130E0C901019687709927D3
:103C80004091840150E08417950709F447C0698387
:103C90007A83FD83EC8396E0929FD001939FB00DD1
:103CA0001124AA57BE4FFE01319601900D929A95AC
:103CB000E1F7809385010E94B11B16E08091840199
:103CC000909185018917C1F1189FC00111248A576D
:103CD0009E4F0E943B1C882379F1E09184011E9F36
:103CE000F0011124EA57FE4F4081518162817381B6
:103CF000848195810E94A11B8091840190E00196AE
:103D00008770992780938401D9CF4F815885698521
:103D10007A858B859C850E94A11BCFCF0E94681B52
:103D20001092850110928401E6EBF1E086E0DF015C
:103D30001D928A95E9F7C1CF2C960FB6F894DEBF95
:103D40000FBECDBFDF91CF911F910895EF92FF92EB
:103D50000F931F93CF93DF938C01892B09F46CC0D1
:103D6000F12CEE24E394E8012196F8018491843744
:103D700040F4843008F051C0813081F0823019F174
:103D80005BC0853709F444C0A8F19CE7980F9037D1
:103D900008F052C08F770E94E21741C00E5F1F4F9C
:103DA000FE01C49180E28C0F883048F4C7708E2DDC
:103DB00001C0880FCA95EAF70E94562114C08C2FC3
:103DC0000E941A172DC00E5F1F4FFE01C49180E2A2
:103DD0008C0F883058F4C7708E2D01C0880FCA959B
:103DE000EAF70E945C210E947D211AC08C2F0E945C
:103DF000E21716C00E5F1F4FFE01C491CC2381F065
:103E00008FE99FE00197F1F700C00000C150F6CFA5
:103E10000E5F1F4FFE01F49003C00E941A178E011F
:103E20008F2D882309F49FCFEFE9FFE03197F1F759
:103E300000C000008150F5CFDF91CF911F910F910D
:103E4000FF90EF90089508956093C0017093C101B1
:103E50008093C2019093C3010C94561B0F931F9340
:103E60000091C0011091C1012091C2013091C301A4
:103E7000DC01CB01802B912BA22BB32B8093C001B3
:103E80009093C101A093C201B093C3011F910F9100
:103E90000C94561B0F931F930091C0011091C10108
:103EA0002091C2013091C301DC01CB018023912319
:103EB000A223B3238093C0019093C101A093C201B8
:103EC000B093C3011F910F910C94561B0F931F9336
:103ED0000091C0011091C1012091C2013091C30134
:103EE000DC01CB0180279127A227B3278093C00153
:103EF0009093C101A093C201B093C3011F910F9190
:103F00000C94561B1092BC011092BD011092BE0180
:103F10001092BF010C94561B41E050E060E070E04D
:103F200004C0440F551F661F771F8A95D2F7409330
:103F3000BC015093BD016093BE017093BF010C940E
:103F4000561B41E050E060E070E004C0440F551F94
:103F5000661F771F8A95D2F78091BC019091BD01B1
:103F6000A091BE01B091BF01482B592B6A2B7B2B2E
:103F70004093BC015093BD016093BE017093BF019B
:103F80000C94561B41E050E060E070E004C0440F28
:103F9000551F661F771F8A95D2F7409550956095FB
:103FA00070958091BC019091BD01A091BE01B0912E
:103FB000BF01482359236A237B234093BC015093BC
:103FC000BD016093BE017093BF010C94561B41E08C
:103FD00050E060E070E004C0440F551F661F771F7B
:103FE0008A95D2F78091BC019091BD01A091BE014C
:103FF000B091BF01482759276A277B274093BC010E
:104000005093BD016093BE017093BF010C94561B89
:104010000F931F930091BC011091BD012091BE012F
:104020003091BF01DC01CB01802B912BA22BB32B54
:104030008093BC019093BD01A093BE01B093BF01DA
:104040001F910F910C94561B0F931F930091BC016D
:104050001091BD012091BE013091BF01DC01CB0167
:1040600080239123A223B3238093BC019093BD01AD
:10407000A093BE01B093BF011F910F910C94561BEA
:104080000F931F930091BC011091BD012091BE01BF
:104090003091BF01DC01CB0180279127A227B327F4
:1040A0008093BC019093BD01A093BE01B093BF016A
:1040B0001F910F910C94561B0895CF92DF92EF92AF
:1040C000FF920F931F93CF93DF938C01C090C00199
:1040D000D090C101E090C201F090C3014091BC01B9
:1040E0005091BD016091BE017091BF01C42AD52AD3
:1040F000E62AF72ACFE1D0E0D701C6010C2E04C092
:10410000B695A795979587950A94D2F780FF07C033
:10411000B8018C2F0E948B0C8130910531F42197CE
:1041200058F7B80180E00E948B0CDF91CF911F916E
:104130000F91FF90EF90DF90CF90089590910C0138
:10414000992321F090910D01911109C020910E0148
:1041500030910F01F90132969FEF40E030C0982F67
:104160009695969596959F30A0F4E0910E01F0916A
:104170000F01E90FF11D877021E030E0A90102C0B5
:10418000440F551F8A95E2F7CA019181892B8183DB
:1041900008959091D70190FF23C01F928F938DEBCC
:1041A00096E09F938F930E9461080F900F900F905D
:1041B0000F9008959F3F39F04F5F4E3041F051917D
:1041C0005813F8CF0DC05111F7CF942FF5CF9F3F63
:1041D00039F0F901E90FF11D97FDFA9582830895F1
:1041E000089590910C01992321F090910D01911166
:1041F00009C020910E0130910F01F9013296205F24
:104200003F4F30C0982F9695969596959F30A8F47D
:10421000E0910E01F0910F01E90FF11D877021E08F
:1042200030E0A90102C0440F551F8A95E2F7CA0188
:10423000809591818923818308959091D70190FF82
:1042400016C01F928F938FE996E09F938F930E94E1
:1042500061080F900F900F900F9008953196E2171C
:10426000F30729F090819813F9CF1082F7CF0895C2
:1042700081E090E0E0910E01F0910F01E80FF91F4D
:104280001082019680319105A9F708959091D60189
:10429000892B8093D601089580959091D60189232A
:1042A0008093D60108951092D60108959091D5017A
:1042B000892B8093D501089580959091D50189230C
:1042C0008093D50108951092D50108958093C4017B
:1042D00008951092C401089580910E0190910F01EC
:1042E000FC0131969C01205F3F4F80E0919191113C
:1042F0008F5FE217F307D1F70895E0910E01F09177
:104300000F018091D6018083E0910E01F0910F01A1
:1043100090818091D501892B80838091C40188236D
:1043200061F0E0910E01F0910F019081892B808363
:104330000E946C2181111092C40180910E01909114
:104340000F010C94981590933B0180933A010895C6
:10435000CF92DF92EF92FF926C01EE24FF24C11402
:10436000D104E104F10421F0C701B60120E101C04C
:1043700020E0C72ED82EE92EFF24C114D104E10479
:10438000F10419F0285FC701B6016B017C0154E00C
:10439000F694E794D794C7945A95D1F7C114D104F1
:1043A000E104F10419F02C5FC701B6016B017C0137
:1043B00042E0F694E794D794C7944A95D1F7C11494
:1043C000D104E104F10419F02E5FC701B601DC014C
:1043D000CB01B695A79597958795892B8A2B8B2B23
:1043E00009F02F5F822FFF90EF90DF90CF9008951C
:1043F0008295982F9C7C392F36953695282F2373DC
:1044000044E0249FC0011124932F982B292F2A7A4E
:104410002695892F8575880F822B08951F93CF933A
:10442000DF931F92CDB7DEB799830E94F821182F32
:104430009981892F0E94F821212F30E0322F2227E5
:10444000A901482BCA010F90DF91CF911F910895C8
:104450008091F001843009F11092D80120E488E1C4
:1044600090E00FB6F894A895809360000FBE20935B
:10447000600083B7817F846083BF83B7816083BF1F
:104480007894889583B78E7F83BF88E10FB6F894C0
:1044900080936000109260000FBE08950895089503
:1044A000CF930E944E220E94300A0E944F22C0E009
:1044B0008C2F0E945C0B811104C0CF5FCE30C1F7FE
:1044C00001C081E0CF9108950E94681B0E948C1565
:1044D0000C94BE0D82E084BD93E095BD9AEF97BD2C
:1044E00080936E0008952FB7F8948091D901909130
:1044F000DA01A091DB01B091DC012FBF0895CF92CA
:10450000DF92EF92FF920F931F932FB7F894409191
:10451000D9015091DA016091DB017091DC012FBF6C
:104520006A017B01EE24FF248C0120E030E0C016FC
:10453000D106E206F30610F4415051099A01281BF6
:10454000390BC9011F910F91FF90EF90DF90CF9031
:1045500008951F920F920FB60F9211248F939F937D
:10456000AF93BF938091D9019091DA01A091DB01C3
:10457000B091DC010196A11DB11D8093D9019093EA
:10458000DA01A093DB01B093DC01BF91AF919F9161
:104590008F910F900FBE0F901F9018950E948A1256
:1045A000F8942FEF87EA91E6215080409040E1F7A0
:1045B00000C0000087E090EBDC018093F90190934C
:1045C000FA01A093FB01B093FC019CE088E10FB6D7
:1045D000F894A895809360000FBE90936000FFCF81
:1045E000EF92FF920F931F93CF93DF93D82FC0E0EA
:1045F0008C2F0E945C0B00E010E0E82EF12CC7012C
:10460000002E02C0959587950A94E2F780FD06C0BA
:104610000F5F1F4F0630110591F709C0602F7C2FE7
:1046200080E00E94690CD813F3CF81E004C0CF5F13
:10463000CE30F1F680E0DF91CF911F910F91FF9086
:10464000EF900895CF93C82F8CE20E94F022882328
:1046500021F08C2FCF910C94F02280E0CF9108951F
:10466000CF930E947F24811102C00E94652482EEB4
:1046700096E00E94C807C5E6C15049F00E94300A82
:104680008FE39CE90197F1F700C00000F5CF8BEDB7
:1046900096E00E94C80789E20E942223811113C17B
:1046A0008AE20E94222381110E94652485E00E94F3
:1046B000222381110E94CE220E948A248093D70156
:1046C00087E00E9422238823A9F18BE10E94222304
:1046D000882351F08091D70181FB222720F991E0B6
:1046E000922790FB81F90EC08EE00E94222388233E
:1046F00061F08091D70182FB222720F991E0922777
:1047000090FB82F98093D70115C080E10E9422239B
:104710009091D701882341F093FB222720F981E073
:10472000822780FB93F904C0892F809580FB90F944
:104730009093D7018091D7010E948E240E949C24DF
:104740008093EA0180EE0E942223882341F0809129
:10475000EA01982F909590FB80F98093EA0189E314
:104760000E942223882359F08091EA0181FB2227AD
:1047700020F991E0922790FB81F98093EA0182EE83
:104780000E942223882359F08091EA0182FB22278C
:1047900020F991E0922790FB82F98093EA0186EE5E
:1047A0000E942223882359F08091EA0183FB22276B
:1047B00020F991E0922790FB83F98093EA0183EE40
:1047C0000E942223882359F08091EA0184FB22274A
:1047D00020F991E0922790FB84F98093EA0185E328
:1047E0000E942223882359F08091EA0185FB222729
:1047F00020F991E0922790FB85F98093EA0181E30B
:104800000E942223882359F08091EA0186FB222707
:1048100020F991E0922790FB86F98093EA0181E1EB
:104820000E942223882359F08091EA0187FB2227E6
:1048300020F991E0922790FB87F98093EA0180911B
:10484000EA010E94A0248091EA0187FB882780F971
:1048500080930D0187E20E942223C82F8EE10E94DF
:1048600022238111C2608FE10E9422238111C46042
:1048700080E20E9422238111C86081E20E942223EB
:104880008111C06182E20E9422238111C06283E211
:104890000E9422238111C06484E20E942223882383
:1048A00011F0C06802C0CC2329F08C2F0E949724FD
:1048B0006C2F03C00E949324682F70E080E090E08A
:1048C000CF910C94241FCF9108956DEE7EEF80E080
:1048D00090E00E94682E60E082E090E00E945A2EF4
:1048E00060E083E090E00E945A2E60E084E090E077
:1048F0000E945A2E60E085E090E00C945A2E80E0F1
:1049000090E00E94542E21E08D3E9E4F09F020E061
:10491000822F089582E090E00C944C2E682F82E064
:1049200090E00C945A2E83E090E00C944C2E682F6B
:1049300083E090E00C945A2E84E090E00C944C2E8E
:10494000682F84E090E00C945A2E8091DF0180FF64
:104950000BC06091130185E0689FB001112475952B
:104960006795759567952BC081FF09C0609113010C
:1049700085E0689FB00111247595679520C082FF7E
:1049800007C06091130185E0689FB001112417C032
:104990009091E0019923D1F060911201961788F768
:1049A0002091130185E0289F90011124929FA0017E
:1049B000939F500D112470E0CA010E941E2E603892
:1049C000710540F46115710539F002C065E070E0D1
:1049D000862F08958FE7089581E008958091DF0183
:1049E00080FF08C06091110170E07595679575951D
:1049F000679521C081FF06C06091110170E0759537
:104A0000679519C082FF04C06091110170E010C069
:104A10009091E0019923C1F0609110019617A0F7E1
:104A200080911101899FC001112470E00E941E2E07
:104A30006038710528F46115710521F0862F0895FD
:104A40008FE7089581E0089561E070E0F4CF803F42
:104A500021F40E94A524819504C0813F29F40E947D
:104A6000A5248093E3010895823F21F40E94A524A8
:104A7000819504C0833F29F40E94A5248093E2011C
:104A80000895893F19F40E94EE2405C08A3F31F44D
:104A90000E94EE2481958093E40108958B3F21F4D8
:104AA0000E94EE24819504C08C3F29F40E94EE24DC
:104AB0008093E5010895843F21F48091E1018160B4
:104AC00017C0853F21F48091E101826011C0863FCB
:104AD00021F48091E10184600BC0873F21F4809133
:104AE000E101886005C0883F31F48091E101806177
:104AF0008093E10108958D3F21F48091DF01816071
:104B00000BC08E3F21F48091DF01826005C08F3F92
:104B100029F48091DF0184608093DF010895803F54
:104B200039F48091E30187FF6CC01092E30169C002
:104B3000813F29F48091E3011816BCF362C0909183
:104B4000E201823F29F497FF5CC01092E20159C054
:104B5000833F19F41916CCF354C0893F41F4809176
:104B6000E40118160CF04DC01092E4014AC08A3FCF
:104B700029F48091E40187FF44C0F6CF8B3F39F4DC
:104B80008091E50187FF3DC01092E5013AC08C3F5E
:104B900029F48091E5011816BCF333C0843F21F459
:104BA0008091E1018E7F17C0853F21F48091E10162
:104BB0008D7F11C0863F21F48091E1018B7F0BC076
:104BC000873F21F48091E101877F05C0883F31F460
:104BD0008091E1018F7E8093E10113C08D3F21F42C
:104BE0008091DF018E7F0BC08E3F21F48091DF0129
:104BF0008D7F05C08F3F29F48091DF018B7F8093EB
:104C0000DF018091E20181110EC08091E3018111E9
:104C10000AC08091E401811106C08091E5018111F3
:104C200002C01092E00108958091D70183FF7EC0F9
:104C30008EE197E00E94C8078091E1011F928F9357
:104C400089E197E09F938F930E94610887E197E045
:104C50000E94C8078091E201282F332727FD309555
:104C60003F938F9384E197E09F938F930E94610815
:104C700082E197E00E94C8078091E301282F332743
:104C800027FD30953F938F938FE097E09F938F930D
:104C90000E9461088DE097E00E94C8078091E401BE
:104CA000282F332727FD30953F938F938AE097E095
:104CB0009F938F930E94610888E097E00E94C80745
:104CC0008091E501282F332727FD30953F938F935F
:104CD00085E097E09F938F930E94610882E097E0C0
:104CE0000E94C8078091E0011F928F938FEF96E09A
:104CF0009F938F930E9461088DEF96E00E94C807F2
:104D00008091DF011F928F938AEF96E09F938F939C
:104D10000E94610887EF96E00E94C8078DB79EB792
:104D20004C960FB6F8949EBF0FBE8DBF81EE91E0FA
:104D30000E94E1150E9473229093DE018093DD01B1
:104D400008951F93CF93DF938091DD019091DE0151
:104D50000E947F22AC019091E001992321F02091E3
:104D6000140130E006C0209115018AE0289F9001CF
:104D700011244217530708F486C08091E201C091C4
:104D8000E301D091E4011091E501811107C0C11147
:104D900076C0D11174C0111172C075C09F3F19F057
:104DA0009F5F9093E001181624F40E94A52480933D
:104DB000E2018091E20187FF05C00E94A524819550
:104DC0008093E2011C1624F40E94A5248093E30141
:104DD0008091E30187FF05C00E94A52481958093FF
:104DE000E3016091E201662339F1C091E301CC2334
:104DF00019F1772767FD7095872F972F0E94232D34
:104E000023E333E343E35FE30E94872D0E94F02C0A
:104E10006093E2016C2F772767FD7095872F972F9E
:104E20000E94232D23E333E343E35FE30E94872DB6
:104E30000E94F02C6093E3011D1624F40E94EE24DE
:104E40008093E4018091E40187FF05C00E94EE2475
:104E500081958093E401111624F40E94EE2480933E
:104E6000E5018091E50187FF05C00E94EE24819550
:104E70008093E501DF91CF911F910C9414269F3F01
:104E800009F08ECF96CFDF91CF911F910895E1EE7B
:104E9000F1E085E0DF011D928A95E9F71092E001CB
:104EA0001092DF01089581E499E00E94C8071F92E3
:104EB00081E08F931F9285E08F9383EF98E09F931B
:104EC0008F930E9461080F900F900F900F900F909A
:104ED0000F9008958330E9F128F4813061F0823039
:104EE00009F10895853009F462C008F449C086309C
:104EF00009F474C0089580911501262F30E0280F21
:104F0000311D2F3F310524F4680F6093150103C054
:104F10008FEF80931501809115011F928F938CE282
:104F200098E072C080911401262F30E0280F311DC7
:104F30002F3F310524F4680F6093140103C08FEFF5
:104F400080931401809114011F928F938AE198E05D
:104F50005BC080911301262F30E0280F311D2F3FB9
:104F6000310524F4680F6093130103C08FEF809321
:104F70001301809113011F928F9387E098E044C042
:104F800080911201262F30E0280F311D2F3F31056F
:104F900024F4680F6093120103C08FEF8093120115
:104FA000809112011F928F9382EF97E02DC0809124
:104FB0001101262F30E0280F311D2F3F310524F439
:104FC000680F6093110103C08FEF809311018091EE
:104FD00011011F928F9389ED97E016C08091100107
:104FE000262F30E0280F311D2F3F310524F4680FA4
:104FF0006093100103C08FEF809310018091100126
:105000001F928F938EEB97E09F938F930E9461087E
:105010000F900F900F900F900895833081F128F436
:10502000813059F08230D1F00895853009F449C0BB
:10503000B8F1863009F456C00895809115016817BB
:1050400020F4861B8093150102C0109215018091F7
:1050500015011F928F938FEA97E054C0809114013D
:10506000681720F4861B8093140102C0109214016B
:10507000809114011F928F938DE997E043C0809136
:105080001301681720F4861B8093130102C010924D
:105090001301809113011F928F938AE897E032C029
:1050A00080911201681720F4861B8093120102C0C0
:1050B00010921201809112011F928F9385E797E061
:1050C00021C080911101681720F4861B8093110183
:1050D00002C010921101809111011F928F938CE5F3
:1050E00097E010C080911001681720F4861B809310
:1050F000100102C010921001809110011F928F9335
:1051000081E497E09F938F930E9461080F900F9026
:105110000F900F900895CF93C82F1F928F9386E41E
:105120009AE09F938F930E94610881E090E0A0E055
:10513000B0E0BC01CD0104C0660F771F881F991F26
:10514000CA95D2F70E94241F0F900F900F900F90D6
:10515000CF910C94681BCF938D3109F465C0B0F5E5
:105160008E3009F4CCC100F5873009F49BC1A8F456
:10517000863009F06DC28091D701817F8E7F809348
:10518000D7018BE49AE00E94C8078DE89EE00E9458
:10519000C80781E08093E70180C1883009F44FC0DF
:1051A0008B3009F47CC154C2863109F4F0C138F463
:1051B000803109F4B8C1813109F430C249C2893162
:1051C00009F4CEC18B3109F486C142C2853309F49A
:1051D00037C248F4873209F433C208F433C2893243
:1051E00009F42EC235C2833438F48A3308F02CC255
:1051F000883309F454C12CC2833409F421C28834A1
:1052000009F026C20E94681B8CE79EE00E94C80736
:105210009FEF23ED80E3915020408040E1F700C0F4
:1052200000000E94CE2239C18CE99EE00E94C8078E
:105230000E94AA2C0E948C150E94BE0D2EC181E9ED
:105240009EE00E94C8078CE59CE00E94C8070E946F
:1052500093241F928F9389E59CE09F938F930E94E4
:10526000610887E59CE00E94C8070E948A24C82F35
:1052700084E49CE00E94C8071F92CF938FE39CE0D8
:105280009F938F930E9461088DE39CE00E94C80762
:1052900083E39CE00E94C8078C2F81701F928F933C
:1052A00080E39CE09F938F930E9461088EE29CE0D4
:1052B0000E94C80784E29CE00E94C807C1FB8827BF
:1052C00080F91F928F9381E29CE09F938F930E94BD
:1052D00061088FE19CE00E94C80783E19CE00E9486
:1052E000C807C2FB882780F91F928F9380E19CE05A
:1052F0009F938F930E9461088EE09CE00E94C807F4
:1053000085E09CE00E94C807C3FBCC27C0F91F9230
:10531000CF9382E09CE09F938F930E94610880E08E
:105320009CE00E94C8070E949C24C82F8CEE9BE042
:105330000E94C8071F92CF9387EE9BE09F938F93A5
:105340000E94610885EE9BE00E94C8078CEC9BE000
:105350000E94C8078C2F81701F928F9389EC9BE06D
:105360009F938F930E9461088DB79EB780960FB66A
:10537000F8949EBF0FBE8DBF87EC9BE00E94C807CC
:1053800080EB9BE00E94C807C1FB882780F91F9231
:105390008F938DEA9BE09F938F930E9461088BEA25
:1053A0009BE00E94C80789E99BE00E94C807C2FBF6
:1053B000882780F91F928F9386E99BE09F938F93B4
:1053C0000E94610884E99BE00E94C80782E89BE094
:1053D0000E94C807C3FB882780F91F928F938FE72D
:1053E0009BE09F938F930E9461088DE79BE00E9452
:1053F000C80783E79BE00E94C807C4FB882780F9A1
:105400001F928F9380E79BE09F938F930E94610888
:105410008EE69BE00E94C8078CE59BE00E94C807CF
:10542000C5FB882780F91F928F9389E59BE09F93A6
:105430008F930E94610887E59BE00E94C8078BE379
:105440009BE00E94C807C6FB882780F91F928F93B4
:1054500088E39BE09F938F930E94610886E39BE023
:105460000E94C8078EE29BE00E94C807C7FBCC27BA
:10547000C0F91F92CF938BE29BE09F938F930E9482
:10548000610889E29BE00E94C8078DB79EB74C96E1
:105490000FB6F8949EBF0FBE8DBFC1E0DEC082E79D
:1054A0009AE05BC08091D701C82FC17080FF09C00E
:1054B0008FE69EE00E94C8078091D701817F8E7F92
:1054C00047C083E69EE00E94C8078091D7018160B3
:1054D0008093D701E2CF9091D70191FBCC27C0F9FF
:1054E00081E0C827892FC0FB81F98093D701CC23A5
:1054F00019F086E59EE027C088E49EE02EC09091DA
:10550000D70192FBCC27C0F981E0C827892FC0FBC7
:1055100082F98093D701CC2319F089E39EE013C070
:1055200089E29EE01AC09091D70193FBCC27C0F985
:1055300081E0C827892FC0FB83F98093D701CC2352
:1055400051F08DE19EE00E94C8078091D7018160F3
:105550008093D70182C080E19EE00E94C8079DCF62
:1055600081E09EE00E94C80785ED9DE00E94C8078B
:1055700088E99DE00E94C8078BE69DE00E94C8076D
:1055800087E29DE00E94C8078CEF9CE0E6CF8EEE9C
:105590009CE00E94C8070E948C151F928F9384ED97
:1055A0009CE09F938F930E94610880910C011F9251
:1055B0008F938DEB9CE09F938F930E946108809165
:1055C0006E011F928F938AEA9CE09F938F930E94B3
:1055D000610880910D011F928F9387E99CE09F9352
:1055E0008F930E9461088091D9019091DA01A09176
:1055F000DB01B091DC01BF93AF939F938F9383E85E
:105600009CE09F938F930E9461088DB79EB746964A
:105610000FB6F8949EBF0FBE8DBF3FCF0E94681B90
:10562000C0910D0181E0C827C0930D01CC2329F062
:1056300089E79CE00E94C80710C08EE69CE08DCFF1
:1056400080E003C08D5101C089530E948B2825CF73
:105650008CE69CE00E94C807C0E08C2FCF91089593
:1056600080E0089580E00895CF93C82F8091E701EE
:10567000813081F020F0823009F44FC045C1E091C3
:105680000E01F0910F018081813169F0823209F0C1
:105690003DC109C0E0910E01F0910F01808181317F
:1056A00011F0823261F48C2F0E94302B811104C0E2
:1056B0008C2F0E94AB282FC081E090E02CC08C2F53
:1056C0000E94322B811126C0C431E1F070F4CB303E
:1056D00081F0C031D1F40E9453278EE39AE00E94FA
:1056E000C80782E08093E70115C0C93259F0C8337A
:1056F00061F48BE49AE00E94C80782E49AE00E9479
:10570000C80708C01092E70103C18CE39AE00E9429
:10571000C807FEC081E08170FDC0C43220F5CE31E3
:1057200008F0C0C0CB3099F1C8F4C73009F0D2C03E
:105730008AE08093150194E19093140193E0909393
:1057400013018093120188E08093110188E2809315
:10575000100182EE98E00E94C807BFC0C33149F132
:10576000C431C1F0B7C0CB3409F4A9C028F4C932A0
:1057700089F0C83361F0AEC0C13509F49EC0C235AE
:1057800009F499C0CE3409F0A5C06AE09EC00E9419
:105790005327A3C08091E601882319F01092E601F7
:1057A0009CC08FEE98E00E94C80781E08093E701DB
:1057B000B1C089EC98E00E94C80787EB98E00E948E
:1057C000C807809115011F928F9384EB98E09F93F7
:1057D0008F930E94610882EB98E00E94C80780EADC
:1057E00098E00E94C807809114011F928F938DE961
:1057F00098E09F938F930E9461088BE998E00E9444
:10580000C8078CE898E00E94C807809113011F9296
:105810008F9389E898E09F938F930E94610887E8AF
:1058200098E00E94C80786E798E00E94C807809128
:1058300012011F928F9383E798E09F938F930E94AA
:10584000610881E798E00E94C8078CE598E00E9413
:10585000C807809111011F928F9389E598E09F936B
:105860008F930E94610887E598E00E94C80780E452
:1058700098E00E94C807809110011F928F938DE3DA
:1058800098E09F938F930E9461088BE398E00E94B9
:10589000C8078DB79EB748960FB6F8949EBF0FBE47
:1058A0008DBF1BC0CE51EC2FF0E0E15DFE4F80813B
:1058B0008093E60112C061E003C061E006C06AE0C7
:1058C0008091E6010E946A2708C08091E6010E944B
:1058D0000D2803C080EE98E013C08091E601882374
:1058E00069F01F928F938AED98E09F938F930E94A7
:1058F00061080F900F900F900F9004C087ED98E013
:105900000E94C80781E006C01092E70180E002C053
:1059100080E001CFCF910895E1E8F0E080818860D8
:1059200080838081816080838FB7F89493E0909327
:10593000890090ED909388008FBF0895EFE6F0E026
:105940008081826080830895EFE6F0E080818D7F22
:1059500080830895EFE6F0E0908182E089278083DC
:1059600008951F920F920FB60F9211242F933F9319
:105970004F935F936F937F938F939F93AF93BF9357
:10598000EF93FF938091E8019091E9010196909344
:10599000E9018093E801811103C082E00E94BE0DFD
:1059A000E091E901E695E695F0E0E455F14FE491E8
:1059B0008091E8018E1303C080E00E94BE0DFF912C
:1059C000EF91BF91AF919F918F917F916F915F9177
:1059D0004F913F912F910F900FBE0F901F901895F0
:1059E00004D06894B1118DC0089570D088F09F578D
:1059F00090F0B92F9927B751A0F0D1F0660F771F1B
:105A0000881F991F1AF0BA95C9F712C0B13081F0FA
:105A100077D0B1E0089574C0672F782F8827B85FDA
:105A200039F0B93FCCF3869577956795B395D9F75B
:105A30003EF490958095709561957F4F8F4F9F4F65
:105A40000895E89409C097FB3EF490958095709571
:105A500061957F4F8F4F9F4F9923A9F0F92F96E9BA
:105A6000BB279395F695879577956795B795F1112F
:105A7000F8CFFAF4BB0F11F460FF1BC06F5F7F4FCC
:105A80008F4F9F4F16C0882311F096E911C07723DE
:105A900021F09EE8872F762F05C0662371F096E8E7
:105AA000862F70E060E02AF09A95660F771F881FB6
:105AB000DAF7880F9695879597F9089557FD9058CE
:105AC000440F551F59F05F3F71F04795880F97FBC2
:105AD000991F61F09F3F79F087950895121613067C
:105AE0001406551FF2CF4695F1DF08C016161706AB
:105AF0001806991FF1CF86957105610508940895E0
:105B0000E894BB2766277727CB0197F908950BD038
:105B100078C069D028F06ED018F0952309F05AC0EB
:105B20005FC01124EECFCADFA0F3959FD1F3950F8C
:105B300050E0551F629FF001729FBB27F00DB11D11
:105B4000639FAA27F00DB11DAA1F649F6627B00DA1
:105B5000A11D661F829F2227B00DA11D621F739F8A
:105B6000B00DA11D621F839FA00D611D221F749F98
:105B70003327A00D611D231F849F600D211D822FDF
:105B8000762F6A2F11249F5750408AF0E1F0882326
:105B90004AF0EE0FFF1FBB1F661F771F881F915033
:105BA0005040A9F79E3F510570F014C0AACF5F3F47
:105BB000ECF3983EDCF3869577956795B795F79566
:105BC000E7959F5FC1F7FE2B880F911D96958795EE
:105BD00097F9089597F99F6780E870E060E008956D
:105BE0009FEF80EC089500240A94161617061806F5
:105BF0000906089500240A941216130614060506D1
:105C00000895092E0394000C11F4882352F0BB0F61
:105C100040F4BF2B11F460FF04C06F5F7F4F8F4FC4
:105C20009F4F0895991B79E004C0991F961708F0BB
:105C3000961B881F7A95C9F78095089597FB072EC4
:105C400016F4009407D077FD09D00E94382E07FC87
:105C500005D03EF4909581959F4F0895709561957C
:105C60007F4F0895EE0FFF1F0590F491E02D0994EA
:105C7000AA1BBB1B51E107C0AA1FBB1FA617B70772
:105C800010F0A61BB70B881F991F5A95A9F780958E
:105C90009095BC01CD010895F999FECF92BD81BDCB
:105CA000F89A992780B50895A8E1B0E042E050E065
:105CB0000C946F2E262FF999FECF1FBA92BD81BD8D
:105CC00020BD0FB6F894FA9AF99A0FBE019608957E
:105CD0000E945A2E272F0C945B2EDC01CB01FC0175
:105CE000F999FECF06C0F2BDE1BDF89A319600B435
:0E5CF0000D9241505040B8F70895F894FFCF40
:105CFE002002BF0DB00E8D0E590E250E0101C501ED
:105D0E0028080A03140A3F4D3620392C06DF05A950
:105D1E000589055005C304DC04F5040E052E0501A6
:0A5D2E00020304050607080900003F
:00000001FF
